:100000000C9462000C948A000C948A000C948A0070
:100010000C948A000C948A000C948A000C948A0038
:100020000C948A000C948A000C948A000C948A0028
:100030000C948A000C948A000C948A000C948A0018
:100040000C942E030C948A000C94B4040C948A0033
:100050000C948A000C948A000C948A000C948A00F8
:100060000C948A000C948A000000000024002700F1
:100070002A0000000000250028002B0000000000DE
:1000800023002600290004040404040404040202DA
:100090000202020203030303030301020408102007
:1000A0004080010204081020010204081020000012
:1000B0000007000201000003040600000000000029
:1000C0000000390611241FBECFEFD4E0DEBFCDBF44
:1000D00011E0A0E0B1E0E2E0F1E102C005900D9294
:1000E000A832B107D9F711E0A8E2B1E001C01D9232
:1000F000A03DB107E1F710E0C4ECD0E004C02297C6
:10010000FE010E947B08C23CD107C9F70E94270369
:100110000C947F080C9400006F927F928F929F92B4
:10012000AF92BF92CF92DF92EF92FF920F931F9305
:1001300080912C0190912D01019709F067C04091A9
:100140002E0150912F01662757FD6095762F8DEB7C
:1001500091E020E030E00E94980760911A017091D0
:100160001B01882777FD8095982F0E9476034EC04B
:10017000232B11F56091180170911901882777FDE3
:100180008095982F0E94760340912E0150912F0167
:10019000662757FD6095762F8DEB91E020E030E0EB
:1001A0000E94980760911A0170911B01882777FDC2
:1001B0008095982F0E94760310932D0100932C01B7
:1001C0008DEB91E00E94FE05909329018093280118
:1001D0008091140161E00E9418044091280150911F
:1001E0002901662757FD6095762F8DEB91E020E081
:1001F00030E00E94980760911A0170911B018827D6
:1002000077FD8095982F0E94760302C001E010E0F0
:100210008DEB91E00E94EA0520912C0130912D0197
:10022000882309F0A5CF2130310509F054C0109280
:100230002B0110922A01BFEF6B2E712C812C912C77
:1002400042C00E94DA03909329018093280100D0D4
:1002500000D0AA2797FDA095BA2FEDB7FEB761820F
:10026000728283829482BC01CD0120E030E040E0C4
:1002700050E0A3EAEA2EA2E0FA2E012D112DAA24C5
:10028000BB2465010E94AD07AB01BC010F900F902C
:100290000F900F908DEB91E020E030E00E949807E6
:1002A00060911A0170911B01882777FD8095982F26
:1002B0000E94760380912A0190912B0101969093E0
:1002C0002B0180932A0180912A0190912B01833088
:1002D00091050CF4B6CF80912C0190912D010197DE
:1002E000F1F584E00E94DA039093290180932801BC
:1002F00000D000D0AA2797FDA095BA2F2FEF30E0AD
:1003000040E050E0EDB7FEB721833283438354834E
:10031000BC01CD0120E030E040E050E0F3EAEF2EF8
:10032000F2E0FF2E012D112DAA24BB2465010E94AD
:10033000AD07AB01BC010F900F900F900F908DEBAC
:1003400091E020E030E00E94980760911A017091DE
:100350001B01882777FD8095982F0E947603809156
:1003600012010E94DA039093290180932801875695
:10037000924024F48091100160E003C0809110014C
:1003800061E00E94180480912C0190912D01019749
:1003900009F047C000D000D0609128017091290178
:1003A000882777FD8095982F2FEF30E040E050E0D0
:1003B000EDB7FEB7218332834383548320E030E0DE
:1003C00040E050E0ECE5EE2EE3E0FE2E012D112D95
:1003D000AA24BB2465010E94AD07AB01BC010F90AC
:1003E0000F900F900F908DEB91E020E030E00E9495
:1003F000980760911A0170911B01882777FD8095FD
:10040000982F0E9476038DEB91E00E94B2066091D6
:100410001A0170911B01882777FD8095982F0E9403
:1004200076031F910F91FF90EF90DF90CF90BF90D8
:10043000AF909F908F907F906F900895EF92FF9272
:100440000F931F93CF93DF938DEB91E040E855E23C
:1004500060E070E00E94F1048091100161E00E9470
:10046000F8038091140161E00E94F8038091160165
:1004700061E00E94F80385E090E008C060E00E941F
:10048000F80380912A0190912B01019690932B0102
:1004900080932A0180912A0190912B018930910546
:1004A0006CF385E090E090932B0180932A0114E097
:1004B000E12EF12C02E010E0C1E0D0E03EC00E944D
:1004C0006504892B89F180912A0190912B01853057
:1004D000910529F4D0932901C093280117C08630D3
:1004E000910529F410932901009328010FC087304A
:1004F000910529F4F0922901E092280107C0883083
:10050000910521F4909329018093280180912E0177
:1005100090912F012091280130912901820F931F82
:1005200090932F0180932E0180912A0190912B01AD
:10053000019690932B0180932A0180912A0190913A
:100540002B01893091050CF4BACF8091140161E040
:100550000E9418046091180170911901882777FD95
:100560008095982F0E9476038DEB91E060E071E01A
:100570000E94AA0660911A0170911B01882777FDDD
:100580008095982F0E9476038DEB91E067E071E0F3
:100590000E94AA0660911A0170911B01882777FDBD
:1005A0008095982F0E9476038DEB91E069E071E0D1
:1005B0000E94AA0660911A0170911B01882777FD9D
:1005C0008095982F0E9476038DEB91E067E071E0B3
:1005D0000E94AA0660911A0170911B01882777FD7D
:1005E0008095982F0E94760360912E0170912F01C3
:1005F0008DEB91E00E94880760911A0170911B01B8
:10060000882777FD8095982F0E94760380911001AE
:1006100061E00E9418048091140160E00E941804B7
:100620008091160161E00E94180468EC70E080E09F
:1006300090E00E9476038091160160E00E94180409
:10064000DF91CF911F910F91FF90EF9008950E943D
:10065000A0030E941E020E948C00FDCF1F920F92E9
:100660000FB60F9211242F933F938F939F93AF93C5
:10067000BF938091340190913501A0913601B091E2
:100680003701309138010196A11DB11D232F2D5F37
:100690002D3720F02D570196A11DB11D2093380153
:1006A0008093340190933501A0933601B0933701C4
:1006B0008091300190913101A0913201B0913301CC
:1006C0000196A11DB11D8093300190933101A0933B
:1006D0003201B0933301BF91AF919F918F913F91C0
:1006E0002F910F900FBE0F901F901895EF92FF92D1
:1006F0000F931F937B018C018FB7F89440913401C5
:100700005091350160913601709137018FBF2FB73D
:10071000F8948091340190913501A0913601B09107
:1007200037012FBF841B950BA60BB70BE816F906F4
:100730000A071B0760F71F910F91FF90EF90089534
:10074000789484B5826084BD84B5816084BD85B5AC
:10075000826085BD85B5816085BDEEE6F0E0808173
:1007600081608083E1E8F0E0808182608083808125
:1007700081608083E0E8F0E0808181608083E1EB4C
:10078000F0E0808184608083E0EBF0E08081816034
:100790008083EAE7F0E080818460808380818260EA
:1007A00080838081816080838081806880831092D3
:1007B000C10008958F7090911C019295990F990F27
:1007C000907C982B90937C0080917A008064809339
:1007D0007A0080917A0086FDFCCF209178004091CC
:1007E0007900942F80E030E0282B392BC90108953F
:1007F000282F30E0C90186569F4FFC0194912A575B
:100800003F4FF9018491882391F0E82FF0E0EE0F3B
:10081000FF1FE859FF4FA591B491662329F48C91ED
:10082000909589238C9308958C91892B8C930895AE
:10083000482F50E0CA0182559F4FFC012491CA0104
:1008400086569F4FFC0194914A575F4FFA013491AD
:100850003323D1F1222331F1233021F48091800020
:100860008F7705C0243031F4809180008F7D809394
:10087000800018C0213019F484B58F7704C022306D
:1008800021F484B58F7D84BD0DC0263021F4809184
:10089000B0008F7705C0273029F48091B0008F7D9C
:1008A0008093B000E32FF0E0EE0FFF1FEE58FF4FF4
:1008B000A591B491662329F48C91909589238C930A
:1008C00008958C91892B8C930895682F70E0CB014B
:1008D00082559F4FFC012491CB0186569F4FFC010E
:1008E00044916A577F4FFB019491992319F420E0BA
:1008F00030E038C0222331F1233021F48091800090
:100900008F7705C0243031F4809180008F7D8093F3
:10091000800018C0213019F484B58F7704C02230CC
:1009200021F484B58F7D84BD0DC0263021F48091E3
:10093000B0008F7705C0273029F48091B0008F7DFB
:100940008093B000892F90E0880F991F84589F4FA3
:10095000FC01A591B4918C9120E030E0842311F04A
:1009600021E030E0C90108951F920F920FB60F9257
:1009700011242F933F934F935F936F937F938F93A4
:100980009F93AF93BF93EF93FF934091C600E09185
:10099000B901F091BA01CF01019660E870E00E94C0
:1009A00015089C018091BB019091BC012817390763
:1009B00039F0E75CFE4F40833093BA012093B901D0
:1009C000FF91EF91BF91AF919F918F917F916F9127
:1009D0005F914F913F912F910F900FBE0F901F90FD
:1009E00018955F926F927F928F929F92AF92BF9273
:1009F000CF92DF92EF92FF920F931F93CF93DF93EB
:100A0000EC013A014B01413482E458078FE068075A
:100A100080E078070CF07FC060E874E88EE190E039
:100A2000A40193010E944A082150304040405040A8
:100A3000CA01B90122E030E040E050E00E944A08DB
:100A400059016A01A6019501209530954095509570
:100A500094E0220F331F441F551F9A95D1F760E091
:100A600074E284EF90E00E944A08CA01B9012FEFB6
:100A700030E040E050E00E94F607A40193010E949C
:100A80004A08C90181509F4F181619061CF4522EAE
:100A90005A9403C055245394521A60E079E08DE3D0
:100AA00090E0A40193010E944A0821503040404048
:100AB0005040CA01B90122E030E040E050E00E941D
:100AC0004A08209530954095509583E0220F331FBA
:100AD000441F551F8A95D1F760E074E284EF90E0DF
:100AE0000E944A08CA01B9012FEF30E040E050E00F
:100AF0000E94F607A40193010E944A08C90181508F
:100B00009F4F181619061CF4822F815002C081E0F5
:100B1000821B851500F5E885F98581E090E00A885B
:100B200002C0880F991F0A94E2F7808360E079E0A1
:100B30008DE390E0A40193010E944A0821503040C7
:100B400040405040CA01B90122E030E040E050E0AE
:100B50000E944A0804C0E885F98510829501EC815D
:100B6000FD813083EE81FF812083EA85FB85208132
:100B700041E050E0CA010E8402C0880F991F0A9418
:100B8000E2F7282B2083EA85FB852081CA010F84A8
:100B900002C0880F991F0A94E2F7282B2083EA8568
:100BA000FB858081088802C0440F551F0A94E2F734
:100BB000842B8083DF91CF911F910F91FF90EF9055
:100BC000DF90CF90BF90AF909F908F907F906F906D
:100BD0005F900895DC011296ED91FC911397E05817
:100BE000FF4F8191919180589F4F20813181821BCD
:100BF000930B60E870E00E9415080895CF93DF938F
:100C0000DC011296ED91FC911397EF01CE57DF4F67
:100C100048815981E058FF4F80819181E058F04030
:100C20008417950719F42FEF3FEF0CC0E40FF51F61
:100C30002081CA01019660E870E00E94150899833E
:100C4000888330E0C901DF91CF910895FC01A08530
:100C5000B18521898C9190E0022E02C095958795EF
:100C60000A94E2F780FFF6CF0484F585E02D6083D7
:100C7000089581E291E09093BE018093BD0189E3E4
:100C800091E09093C0018093BF0185EC90E0909338
:100C9000C2018093C10184EC90E09093C4018093E1
:100CA000C30180EC90E09093C6018093C50181EC74
:100CB00090E09093C8018093C70186EC90E09093F8
:100CC000CA018093C90184E08093CB0183E08093C3
:100CD000CC0187E08093CD0185E08093CE0181E057
:100CE0008093CF0108950F931F93CF93DF938C01CF
:100CF000EB0109C02196D801ED91FC910190F081A2
:100D0000E02DC801099568816623A1F7DF91CF9195
:100D10001F910F910895EF92FF920F931F93CF931E
:100D2000DF938C017B01EA010CC0D7016D917D013D
:100D3000D801ED91FC910190F081E02DC801099559
:100D40002197209791F7DF91CF911F910F91FF90FD
:100D5000EF900895DC01ED91FC910280F381E02D8C
:100D6000099508950F931F938C01DC01ED91FC917F
:100D70000190F081E02D6DE00995D801ED91FC9195
:100D80000190F081E02DC8016AE009951F910F9153
:100D900008952F923F924F925F926F927F928F921F
:100DA0009F92AF92BF92CF92DF92EF92FF920F93FA
:100DB0001F93DF93CF93CDB7DEB7A0970FB6F8940C
:100DC000DEBF0FBECDBF1C016A017B01411551057D
:100DD0006105710549F4DC01ED91FC910190F08110
:100DE000E02D60E3099554C0882499245401422ED3
:100DF00055246624772401E010E00C0F1D1F080D18
:100E0000191DC701B601A30192010E942808F8012B
:100E100060830894811C911CA11CB11CC701B60100
:100E2000A30192010E942808C901DA016C017D0129
:100E3000C114D104E104F104F1F681E0E82EF12CB3
:100E4000EC0EFD1EE80CF91C3E010894611C711C9F
:100E5000D501C4010197A109B1096C01C818D908CD
:100E600014C0F601EE0DFF1D60816A3010F4605D64
:100E700001C0695CD101ED91FC910190F081E02D00
:100E8000C10109950894E108F1086E147F0449F73F
:100E9000A0960FB6F894DEBF0FBECDBFCF91DF9105
:100EA0001F910F91FF90EF90DF90CF90BF90AF9088
:100EB0009F908F907F906F905F904F903F902F907A
:100EC0000895EF92FF920F931F93CF93DF93EC015E
:100ED0007A018B0177FF0FC0E881F9810190F081E1
:100EE000E02D6DE2099510950095F094E094E11CD9
:100EF000F11C011D111DCE01B801A7012AE00E94BD
:100F0000C906DF91CF911F910F91FF90EF90089547
:100F10000F931F938C01AB01662757FD6095762FC9
:100F20000E946107C8010E94B2061F910F910895A7
:100F3000DC012115310541F4ED91FC910190F08126
:100F4000E02D642F099508952A30310519F40E9487
:100F5000610708950E94C90608952F923F924F920B
:100F60005F926F927F928F929F92AF92BF92CF9239
:100F7000DF92EF92FF920F931F93DF93CF93CDB742
:100F8000DEB73B014C0119012A016D897E898F89E9
:100F9000988D6A197B098C099D09621A730A840A63
:100FA000950AA40193010E94F607E218F3080409C8
:100FB0001509A80197010E944A082A0D3B1D4C1DE6
:100FC0005D1DB901CA01CF91DF911F910F91FF9073
:100FD000EF90DF90CF90BF90AF909F908F907F90D9
:100FE0006F905F904F903F902F900895629FD00137
:100FF000739FF001829FE00DF11D649FE00DF11DD4
:10100000929FF00D839FF00D749FF00D659FF00D82
:101010009927729FB00DE11DF91F639FB00DE11D6F
:10102000F91FBD01CF011124089597FB092E072652
:101030000AD077FD04D049D006D000201AF470956C
:1010400061957F4F0895F6F7909581959F4F08958C
:10105000A1E21A2EAA1BBB1BFD010DC0AA1FBB1FBC
:10106000EE1FFF1FA217B307E407F50720F0A21B2E
:10107000B30BE40BF50B661F771F881F991F1A949B
:1010800069F760957095809590959B01AC01BD01C5
:10109000CF01089597FB092E05260ED057FD04D0E9
:1010A000D7DF0AD0001C38F4509540953095219533
:1010B0003F4F4F4F5F4F0895F6F79095809570958D
:1010C00061957F4F8F4F9F4F0895AA1BBB1B51E126
:1010D00007C0AA1FBB1FA617B70710F0A61BB70BA8
:1010E000881F991F5A95A9F780959095BC01CD014D
:1010F0000895EE0FFF1F0590F491E02D0994F894E8
:02110000FFCF1F
:10110200536F7920656C002000487962726964002F
:101112000D00030004000900140003000100000098
:0811220000260673068B06008F
:00000001FF
